:100000000C9430010C944D010C9468010C944D013A
:100010000C944D010C944D010C944D010C944D0128
:100020000C944D010C944D010C9422190C944D012B
:100030000C944D010C944D010C944D010C944D0108
:100040000C944D010C944D010C944D010C944D01F8
:100050000C944D015705570583058305E5050306F7
:100060001B071B070E06A706B806B80629003A00AC
:100070003B003C003D003E003F004000410042008C
:1000800043004400450046004C0035001E001F00A0
:100090002000210022002300240025002600270044
:1000A0002D002E002A004A002B0014001A00080020
:1000B000150017001C0018000C00120013002F0080
:1000C000300031004B003900040016000700090021
:1000D0000A000B000D000E000F003300340000007A
:1000E00028004E00E1001D001B000600190005005D
:1000F00011001000360037003800E5000000520003
:100100004D00E0000000E300E20000002C000000D1
:1001100000000000E600E4000000500051004F0025
:1001200009023B00020100A0FA09040000010301DA
:100130000100092101010001224000070581030897
:100140000001090401000103000000092101010070
:1001500001227B0007058303080001120110010042
:100160000000086BB1E50412000102000118034809
:100170000065007200720069006E00670062006F27
:10018000006E00650000001803520061006D006FF2
:10019000006E00200049006D00620061006F0000E9
:1001A000000403090405010902A10185020901A156
:1001B0000005091901290815002501950875018117
:1001C000020501093009311581257F9502750881E5
:1001D0000609381581257F950175088106050C0AE9
:1001E00038021581257F950175088106C0C005017B
:1001F0000980A101850319012AB700150126B7005E
:10020000950175108100C0050C0901A10185041933
:10021000012AA002150126A002950175108100C0D7
:1002200005010906A101050719E029E715002501C7
:10023000950875018102950175088103050719006C
:1002400029FF150026FF009506750881000508198D
:10025000012905950575019102950175039103C06A
:1002600011241FBECFE5D8E0DEBFCDBF10E0A0E671
:10027000B0E0E0EBF9E302C005900D92A23FB107B8
:10028000D9F722E0A2EFB0E001C01D92AB3BB2076C
:10029000E1F70E944D130C94D61C0C940000A82F7B
:1002A000B92F80E090E041E050EA609530E009C06D
:1002B0002D9182279795879510F084279527305E9A
:1002C000C8F36F5FA8F30895EADF8D939D930895B7
:1002D000CF93CFB7CF93DF93C395839BE9F7839BEE
:1002E00010C0839B0EC0839B0CC0839B0AC0839B62
:1002F00008C0839B06C0C0919202C395C09392022E
:100300008EC06F93C0919102DD27C756DD4F2F93AA
:1003100065E5839B03C02F916F91E1CF0F931F93EE
:100320004F9320E040E15F9300B30C7003FB27F98B
:100330003F9350E03BE039C01C7040642F77012FA1
:100340005F5F1EC0406810B31C702F7752501FC0F3
:10035000406400B32F770C70D1F15F5F00C023C001
:10036000406210B32F771C7091F15F5F00C025C011
:100370000C701027515012F45D5F0000115027954A
:100380002C3F10B3C8F61C700127015027952C3F55
:10039000C8F64227499300B30C7010274F731150D1
:1003A00027952C3FA8F64695469510B31C7079F01A
:1003B0000127015027952C3F98F66B5A60F3315076
:1003C00000B3B0F600C010E81ABF00271CC03B50B5
:1003D0003195C31BD04010E81ABF0881033C21F1BE
:1003E0000B3411F120918E021981110F1213EDCFF0
:1003F0004A81441F093679F10D3211F0013E29F787
:100400004F7009F0042F009397023F915F914F9135
:100410001F910F912F916F91CAB7C7FD5DCFDF91EB
:10042000CF91CFBFCF91189520919702222369F3E6
:1004300010919502112309F049C034300AF448C0E4
:100440003093950220939002109191023BE0311B72
:10045000309391023DC0009195020130BCF50AE550
:100460004F7049F43091790034FD33C00093790026
:10047000CBE6D2E032C0433059F0443091F03091B5
:10048000760234FD26C000937602C7E7D2E025C08D
:100490003091AF0234FD1DC00093AF02C0EBD2E03B
:1004A0001CC03091820234FD14C000938202C3E864
:1004B000D2E013C0052710E000C0000002BB1AC044
:1004C000052710E0221F1DC010E021C04AE502C030
:1004D00032ED432FC4E1D0E032E011B31C60939AB7
:1004E00002B311BB5CE020E865E320FF052702BBF7
:1004F000279517951C3FF0F66695B8F7B1F720FFE2
:10050000052702BB279517951C3FD0F62795179511
:1005100017FF052700001C3F02BBB0F629913A9552
:1005200019F7037F10919602110FC651D04002BBFC
:1005300011F010938E0210E81ABF086011B3137FF8
:10054000402F437F54E05A95F1F702BB11BB42BBE9
:100550005CCF81E0089581E008950C94AB0208958A
:100560000C94AF021F93CF93DF9300D000D01F9263
:10057000CDB7DEB749835A836B833091F50089810B
:100580009A81311114C0662359F0222349F00E9448
:100590005809182F682F89819A810E94010903C088
:1005A0000E942C09182F69817A81812F04C00E9432
:1005B000580969817A810F900F900F900F900F90DA
:1005C000DF91CF911F910C94BE10FC01262F40812A
:1005D00051816281738184810C94B20281E008951B
:1005E000CF93DF93EC0160E00E94E502BE01DF9152
:1005F000CF910C94B0020C9404120C940012089544
:100600000E94AB070E94FF022FEF84E39CE0215081
:1006100080409040E1F700C000000C9448190F930F
:100620001F93CF93DF938C0161E00E94E502EC0100
:10063000B8010E94AD028823F1F1B801CE010E94F9
:10064000CF178823C1F1B801CE010E94E31588239A
:1006500091F1B801CE010E942B17882361F1F801B6
:100660008281882309F1CB358DE5D807C1F050F49C
:10067000C115FCE5DF0781F0CF3DDC45A9F40E9400
:10068000BF0E19C0CC35EDE5DE0761F0CD35DD4597
:1006900059F40E94020E08C00E9400030CC00E9480
:1006A0000B0E02C00E940E0EC801DF91CF911F9168
:1006B0000F910C94A90280E0DF91CF911F910F91CF
:1006C00008950E94CC180C947A030E947D030C9428
:1006D000D21808950C94690381E008950C946C037A
:1006E0000895CF93C82F0E946A038C2F0E946E0337
:1006F000CF91089580E00C9471030E942B180C9404
:1007000071030E942B189091F400891721F08093B7
:10071000F4000C9471030895CF93DF93CDB7DEB747
:100720002B970FB6F894DEBF0FBECDBF4F8358870F
:1007300069877A878B8761110E944E0D9E012F5F1A
:100740003F4F86E0F90111928A95E9F785E0FE01B5
:100750003796D90101900D928A95E1F789819A81A6
:100760004C815D81452B31F09F3F31F491E08F3F0B
:1007700019F403C091E001C090E090FF09C04981E5
:100780005A816B817C818D819E810E946F0C05C096
:10079000C9010E94EE028111F2CF2B960FB6F89498
:1007A000DEBF0FBECDBFDF91CF910895FC018081E8
:1007B00091810E949A090895CF93882309F4A4C0D7
:1007C000C82F8238C1F40E942B1881FD9DC069E3B7
:1007D00080916200909163000E94BE180E94700D8B
:1007E0002FEF81EE94E0215080409040E1F700C06F
:1007F000000069E319C0833801F50E942B1880FDC1
:1008000083C063E580916200909163000E94BE18EE
:100810000E94700D2FEF81EE94E0215080409040B7
:10082000E1F700C0000063E58091620090916300F1
:100830000E94C018CF910C94700D8438C1F40E94AE
:100840002B1882FD61C067E4809162009091630083
:100850000E94BE180E94700D2FEF81EE94E021508F
:1008600080409040E1F700C0000067E4DDCF8CEFEE
:100870008C0F813AD0F46C2F8091620090916300CC
:100880000E948818882349F06C2F80916200909113
:1008900063000E94C0180E94700D6C2F809162004E
:1008A000909163000E94BE18C5CF80E28C0F883003
:1008B00048F4C77081E001C0880FCA95EAF70E942A
:1008C000310DB8CFEBE5EC0FE33040F4F0E0E85544
:1008D000FF4F808190E0CF910C945018E8E5EC0F29
:1008E000E73150F4F0E0EE0FFF1FE658FF4F808134
:1008F0009181CF910C946618CD3E30F08C2F0E94E0
:10090000D213CF910C94A414CF910895882309F4A5
:1009100064C0823879F40E942B1881FF5EC069E3BD
:1009200080916200909163000E94BE180E94700D39
:1009300069E310C08338B1F40E942B1880FF4DC0CA
:1009400063E580916200909163000E94BE180E944E
:10095000700D63E580916200909163000E94C01861
:100960000C94700D843879F40E942B1882FF35C0E6
:1009700067E480916200909163000E94BE180E941B
:10098000700D67E4E7CF9CEF980F913A10F4682F51
:10099000E1CF90E2980F983050F4877091E001C059
:1009A000990F8A95EAF7892F0E94370DD9CF9BE5D9
:1009B000980F933020F480E090E00C94501898E564
:1009C000980F973120F480E090E00C9466188D3EEB
:1009D00020F00E942D140C94A41408951F93CF931B
:1009E000DF93182FEB010E94DC03209741F08FE981
:1009F0009FE00197F1F700C000002197F6CF812F0B
:100A0000DF91CF911F910C948604893319F060E037
:100A100070E002C060E570E00C94EE04882321F0E1
:100A20000E94310D0C94700D0895882321F00E94CE
:100A3000370D0C94700D0895CF92DF92EF92FF92D4
:100A40000F931F93CF93DF937C01D62FC72FFC0109
:100A50001281058102950F700E94270D8823B9F03D
:100A60001123A9F08C2F807F803421F080E28D0F3C
:100A7000883068F080914E0282FD09C082E00E94B9
:100A8000D00D0E94270D91E0D82ED92601C0D12C7F
:100A9000CC2EC2948FE0C8228C2D90E08C30910532
:100AA00008F0C9C1FC01E65DFF4F0C946E1C8C2F51
:100AB000807FCF70882311F0C295C07F112399F0F9
:100AC000CC2309F4A4C180E28D0F883010F0D1113D
:100AD00004C08C2F0E94310D03C08C2F0E94410D49
:100AE0000E94700D94C18D2F0E948604CC2309F4BE
:100AF000A2C180E28D0F883038F1DD2329F18C2FDF
:100B00000E94470D24C08C2F807FCF70803211F05F
:100B1000C295C07FDD2319F0D130A1F140C0809192
:100B20004E0282FF17C0112349F0CC2329F08C2FED
:100B30000E94310D0E94700D80E06AC180E00E9429
:100B40008604CC2309F477C18C2F0E94370D0E94B4
:100B5000700D71C1112371F0002341F0013031F4A7
:100B60000E94510D8C2B0E94590D65C10E94510DA0
:100B70008C2B0EC0002319F0013009F45CC10E94D7
:100B8000660D1FC0112339F0063008F054C18C2FB8
:100B90000E940E0550C1053008F04DC112C011234E
:100BA00019F00023A1F333C1002359F0D93309F020
:100BB0003FC1FFEF07EE13E0F15000401040E1F7B6
:100BC00035C18C2F0E94150536C18C2F86958695D0
:100BD000837019F0813061F02EC1112321F08D2F27
:100BE0009C2F937002C080E090E00E9450182BC1AF
:100BF000112321F08D2F9C2F937002C080E090E094
:100C00000E94661820C18D2F112319F00E94D21363
:100C100002C00E942D140E94A41415C18C2F837051
:100C200009F047C011110BC12D2F22952695277071
:100C3000220F220F6D2F6F70862F90E0A0E0B0E0A2
:100C4000022E04C0880F991FAA1FBB1F0A94D2F757
:100C5000D4FF10C04FE050E060E070E004C0440FEB
:100C6000551F661F771F2A95D2F7409550956095BE
:100C7000709503C040E050E0BA01C695C695C370B8
:100C80008A019B01082B192B2A2B3B2BC901B80188
:100C9000C23049F058F4C13019F00E941708CFC093
:100CA0000E940508CCC00E942908C9C00E94030800
:100CB000C6C0112319F08C2F817001C0869588233E
:100CC00009F4BDC02D2F229526952770220F220FE3
:100CD0006D2F6F70862F90E0A0E0B0E0022E04C070
:100CE000880F991FAA1FBB1F0A94D2F7D4FF10C008
:100CF0004FE050E060E070E004C0440F551F661FF5
:100D0000771F2A95D2F7409550956095709503C04E
:100D100040E050E0BA01C695C695C3708A019B01B8
:100D2000082B192B2A2B3B2BC901B801C23049F0E3
:100D300058F4C13019F00E94DC0881C00E94CA0832
:100D40007EC00E94EE087BC00E943D0878C0CF7034
:100D5000112339F08C2F0E9463088D2F0E940E05FD
:100D60006EC08D2F0E9415058C2F0E94840867C0CD
:100D7000D23F21F128F4D03F41F0D13FC1F043C030
:100D8000D33F19F1D43F79F03EC0112341F0053033
:100D900008F051C08C2F8F710E94A9084CC00630FA
:100DA00008F049C0F7CF80914E0282FF18C011238E
:100DB00039F08C2F8F710E9463083DC01123C9F355
:100DC0008C2F8F710E94840836C0112329F08C2F3C
:100DD0008F710E944E082FC00E9449082CC0112319
:100DE00049F0CF718C2F0E94630863E08C2F0E9422
:100DF000B50D21C081E00E94D00D0230E0F082E00C
:100E00000E94D00D18C0112331F0002391F28D2FD4
:100E10000E94DC0310C0002399F2D93349F41FEF7C
:100E200027EE33E0115020403040E1F700C00000D1
:100E30008D2F0E94860488EF8C0D843020F40E9450
:100E40002B180E947103DD20C9F00E94230D80FD44
:100E500015C0F70112820E941D0D0E946308C70190
:100E60000E945F070E941D0DDF91CF911F910F918E
:100E7000FF90EF90DF90CF900C948408DF91CF919A
:100E80001F910F91FF90EF90DF90CF9008950F93F7
:100E90001F93CF93DF93EC01688179818A810E944F
:100EA000A5098C010E9400090E94F107B801CE013A
:100EB0000E941C05DF91CF911F910F910895CF9350
:100EC000DF93EC01988189812B813C81232B31F0C8
:100ED0008F3F31F481E09F3F19F403C081E001C0EE
:100EE00080E080FD1DC0CE010E940F03811110C063
:100EF0000E94270D8823A1F08A81882389F08091A0
:100F00004E0282FD0DC082E0DF91CF910C94D00D96
:100F1000CE010E944707CE01DF91CF910C94F002E1
:100F2000DF91CF91089580E090E00E94501880E01A
:100F300090E00E9466180E944E0D0E94700D0E9463
:100F4000D5150C94A41480916200909163000E94C6
:100F5000C2180C9493070E943E0D0C94A30792951F
:100F60009F70963079F010F4925001C09A509230F0
:100F700068F4803F69F018F4883E40F409C0843F6B
:100F800029F406C0883E20F0813F11F080E00895EA
:100F900081E00895FC01808191810E949A090E945C
:100FA000AF070895CF93DF9300D000D01F92CDB745
:100FB000DEB70F900F900F900F900F90DF91CF91B1
:100FC0000895CF93DF9300D000D000D0CDB7DEB727
:100FD00026960FB6F894DEBF0FBECDBFDF91CF913E
:100FE0000895089508950C94F2070C94F3070E9455
:100FF000F507609336017093370180933801909321
:1010000039010C9493070C94F7070F931F930091E9
:101010003601109137012091380130913901602B50
:10102000712B822B932B1F910F910C94F7070F9329
:101030001F930091360110913701209138013091B2
:10104000390160237123822393231F910F910C9404
:10105000F7070F931F9300913601109137012091EC
:1010600038013091390160277127822793271F911A
:101070000F910C94F7070C94F2070E943B086093C1
:1010800032017093330180933401909335010C94B5
:10109000930760E070E0CB010C943D080F931F9321
:1010A00041E050E060E070E08A019B0104C0000F65
:1010B000111F221F331F8A95D2F7C901B8011F9152
:1010C0000F910C943D080F931F9341E050E060E0B6
:1010D00070E004C0440F551F661F771F8A95D2F732
:1010E0008091320190913301A0913401B09135018A
:1010F0008A019B01082B192B2A2B3B2BC901B80114
:101100001F910F910C943D080F931F9341E050E005
:1011100060E070E004C0440F551F661F771F8A957A
:10112000D2F74095509560957095809132019091DD
:101130003301A0913401B09135018A019B0108234C
:1011400019232A233B23C901B8011F910F910C9445
:101150003D080F931F9341E050E060E070E004C051
:10116000440F551F661F771F8A95D2F78091320171
:1011700090913301A0913401B09135018A019B0116
:10118000082719272A273B27C901B8011F910F916A
:101190000C943D080F931F9300913201109133017D
:1011A0002091340130913501602B712B822B932BD0
:1011B0001F910F910C943D080F931F9300913201E2
:1011C0001091330120913401309135016023712356
:1011D000822393231F910F910C943D080F931F932B
:1011E0000091320110913301209134013091350189
:1011F00060277127822793271F910F910C943D0838
:1012000008952FE0929F800D1124E82FE695E69532
:10121000E695877051E001C0550F8A95EAF785E0A1
:10122000E89FF0011124EA50FF4F20E030E070E029
:101230004081CB01022E02C0969587950A94E2F771
:101240008170819584278523842781932F5F3F4F69
:101250002530310569F708952FE0929F800D112404
:10126000682F669566956695982F977085E0689FBC
:10127000B001112440E050E080E0FB01E40FF51FD5
:10128000EA50FF4F208130E0092E02C036952795A5
:101290000A94E2F721703327042E01C0220F0A942A
:1012A000EAF7822B4F5F5F4F4530510531F70895C4
:1012B000BF92CF92DF92EF92FF920F931F93CF9343
:1012C000DF938C01C0903201D0903301E090340163
:1012D000F09035018091360190913701A09138014D
:1012E000B0913901C82AD92AEA2AFB2ACFE1D0E0F5
:1012F000D701C6010C2E04C0B695A7959795879582
:101300000A94D2F780FD04C0219790F7B12C07C052
:10131000BC2EB8018C2F0E94D1100197A9F38B2D00
:10132000DF91CF911F910F91FF90EF90DF90CF90C1
:10133000BF900895CF93DF93EC010E945809BE013E
:101340000E94D110DF91CF9108951F93CF93DF9327
:10135000EB019091F500992321F0CB010E949A09AD
:1013600013C0882349F0CB010E945809182F682F19
:10137000CE010E94010904C0CB010E942C09182F44
:10138000BE01812F0E94D110DF91CF911F9108954E
:101390001F93CF93DF93C0913A0116E080913B01F8
:1013A000C81799F0D0E01C9FF0011D9FF00D11248B
:1013B000E45CFE4F4081518162817381848195811B
:1013C0000E94E1072196C770E9CFDF91CF911F916D
:1013D000089540916C0150916D0160916E01709182
:1013E0006F0180917001909171010C94E10720913F
:1013F0003A0190913B0156E02917A9F030E0529F45
:10140000F001539FF00D1124E45CFE4F71817613BF
:1014100006C07081781303C07281741306C02F5FF9
:101420003F4F2770E9CF80E0089581E00895EF9263
:10143000FF920F931F93CF93DF9380917101829559
:101440008F7009F065C080916E01882309F460C037
:1014500080913A01F0903B0110916C0100916D0177
:1014600060916F017091700191E01F3F09F090E071
:10147000C0916000D0916100292F96E0E92E8F1570
:1014800009F446C06115710521F00F3F21F030E0ED
:1014900003C031E001C0322F90E030FD36C0E89E3D
:1014A000F001E99EF00D1124DF01A45CBE4F1196FE
:1014B0003C911197301329C03C91311326C01296EC
:1014C0003C911297311121C013964D915C91149764
:1014D000461B570B4C175D07C0F4809171018F704C
:1014E000806180937101EF5BFE4F80818F7080611E
:1014F00080838CE691E00E945F07DF91CF911F917E
:101500000F91FF90EF900C94C80901968770B7CFA8
:10151000DF91CF911F910F91FF90EF9008958F92DF
:101520009F92AF92BF92CF92DF92EF92FF920F9372
:101530001F93CF93DF93CDB7DEB761970FB6F894C3
:10154000DEBF0FBECDBF8C0185E0F801DE011D9628
:1015500001900D928A95E1F7D8011296EC90909146
:101560006C0120916D0140916F0150917001411506
:10157000510531F02F3F31F481E09F3F19F403C052
:1015800081E001C080E080FD7CC1F801C080D18095
:10159000838094808CE6A82E81E0B82EF0906E01B6
:1015A000B401641B750B4091600050916100FF20F5
:1015B00009F411C180917101382F307F64177507CC
:1015C00008F0CBC031118AC0D21214C0C91212C0A7
:1015D000FE2CE1100FC08F708061809371010E941A
:1015E000E909C5010E945F0780917101D801159634
:1015F0008C9361C18114910439F0BFEFDB1206C0F6
:1016000081E0CB1203C003C081E001C080E080FD17
:1016100003C081E08E2502C080E090E080FF10C012
:101620004E2D6D2D8C2D0E94F709882349F08CE6F4
:1016300091E00E945F07ECE6F1E086E0DF019DC0EB
:10164000892839F0BFEFDB1206C081E0CB1203C05E
:1016500003C081E001C080E080FD03C081E08E25F1
:1016600002C080E090E0E82FE170BE2E80FF2CC029
:101670004E2D6D2D8C2D0E94F709F82E811124C05E
:10168000CD86DE868D859E850E949A09292F22951A
:101690002F70223018F0243090F405C09F7059F05C
:1016A000811109C008C19F7031F0D80115969C9135
:1016B000907F09F400C1805E883008F4FCC0C80146
:1016C0000E945F07FB2CF7C0FE2CEE2009F4F3C04C
:1016D0008091710181608093710154C0D21206C063
:1016E000C91204C0E11002C0F80199C0C8010E94EB
:1016F000CA07882361F1EE2051F120917101822FF8
:1017000082958F7090E0029774F080916C019091B7
:101710006D0198878F8319869B868A862C87CE01D8
:1017200007960E945F0786E0F801ACE6B1E0019001
:101730000D928A95E1F70E94170A0E94E9090AC0F2
:10174000D21611F1C8010E94CA0781112CC0C8012C
:101750000E945F07FF24F394AEC03111F1CF782DC2
:10176000998A888AA6016E2D89890E94D2078CE603
:1017700091E00E945F0786E0D5011D928A95E9F706
:101780000E94E909F12C97C0C912DCCFE110DACF31
:10179000F8018583C8010E945F0786E0D5011D928C
:1017A0008A95E9F788C0EE2091F220917101822F8D
:1017B00082958F7090E002970CF4B5CF80916C0108
:1017C00090916D019A8389831B829D828C822E83E6
:1017D000CE010196A6CF6417750708F044C0FE2C11
:1017E000EE2009F4B4CFD21230C0C9122EC020911D
:1017F000710120FD21C0822F82958F70482F50E00B
:1018000041155105C9F0F80125834F30510541F0CC
:101810008F5F982F9295907F822F8F70892B858371
:10182000C8010E945F0786E0F801ACE6B1E00190D4
:101830000D928A95E1F73DC086E0F801ACE6B1E093
:1018400001900D928A95E1F736C0C8010E94CA073F
:10185000811169CF80917101816080937101C8010C
:101860000E945F0728C0782D998A888AA6016E2D6C
:1018700089890E94D20786E0D5011D928A95E9F7F1
:1018800018C0EE2009F463CFC8010E94CA07F82EE1
:10189000882309F45CCF86E0F801ACE6B1E0019062
:1018A0000D928A95E1F78CE691E00E94D6030E94A2
:1018B000170A0E94E9098F2D61960FB6F894DEBFD2
:1018C0000FBECDBFDF91CF911F910F91FF90EF9091
:1018D000DF90CF90BF90AF909F908F9008951F930F
:1018E000CF93DF93CDB7DEB72C970FB6F894DEBF5A
:1018F0000FBECDBF4F83588769877A878B879C87B8
:10190000CE0107960E948F0A8823D1F09F81888597
:101910002A853B85232B31F08F3F31F481E09F3FB7
:1019200019F403C081E001C080E080FD47C04F8111
:10193000588569857A858B859C850E94E1073EC024
:1019400086E0FE013796DE01119601900D928A9590
:10195000E1F7FF81E8856A857B856115710531F0C6
:10196000EF3F31F481E0FF3F19F403C081E001C093
:1019700080E080FD23C020913B0130E0C901019649
:101980008770992740913A0150E084179507F1F14B
:10199000F983EA837D836C8396E0929FD001939FC5
:1019A000B00D1124A45CBE4FFE01319601900D9242
:1019B0009A95E1F780933B010E94C80916E0809157
:1019C0003A0190913B01891771F1189FC0011124D0
:1019D000845C9E4F0E948F0A882329F1E0913A018E
:1019E0001E9FF0011124E45CFE4F40815181628111
:1019F0007381848195810E94E10780913A0190E092
:101A000001968770992780933A01D9CF0E94AB073E
:101A100010923B0110923A01ECE6F1E086E0DF0122
:101A20001D928A95E9F72C960FB6F894DEBF0FBE8B
:101A3000CDBFDF91CF911F91089580917A01859557
:101A400085958595089580917A0187700895909184
:101A50007A01977081E009F480E008958091850112
:101A6000089590918501892B809385010895809533
:101A700090918501892380938501089510928501B5
:101A8000089590918401892B809384010895809515
:101A90009091840189238093840108951092840198
:101AA000089580917B01089508950C94540D0C9431
:101AB000550D90914E0292FD08C090917B019817B0
:101AC00021F080937B010C94570D089580917B0148
:101AD000882329F010927B0180E00C94570D089523
:101AE000CF93DF93E0916200F091630080918501D4
:101AF0008083E0916200F091630090818091840185
:101B0000892B808380917B01882381F0E0916200A2
:101B1000F09163009081892B808380916200909185
:101B200063000E947C1881110E94660DC0916200C2
:101B3000D091630048E050E062E771E0CE010E947E
:101B4000881C892B69F088E0FE01A2E7B1E00190D2
:101B50000D928A95E1F7CE01DF91CF910C94371861
:101B6000DF91CF9108950C94540D90914E0292FD07
:101B700010C098E0899F90011124262B20937A01B0
:101B80000E94630880917A018595859585950C94CE
:101B9000B30D0C94630810927A0180E00C94B30D9D
:101BA00020917A018095822380937A01982F9770F3
:101BB00099F430E0482F082E000C550B24173507F8
:101BC00059F090914E0292FD07C0859585958595B7
:101BD0000E9484080C94CB0D089590914E0292FBC4
:101BE000222720F9281769F080FB92F990934E0282
:101BF00080914D0290914E020E943B0E82E00C9427
:101C0000D00D089580914E0282FB882780F991E0E3
:101C100089270C94ED0D81E00C94ED0D80E00C947F
:101C2000ED0D6FEF7FEF80E090E00C94C01C80E042
:101C300090E00E949D1C21E0893E9E4F09F020E02B
:101C4000822F089582E090E00C94951C83E090E050
:101C50000C94951CCF9384E090E00E94951CC82FB3
:101C600082E290E00E94951C2C2F30E0A901582BB5
:101C7000CA01CF910895CF93C92F682F84E090E0D7
:101C80000E94A31C6C2F82E290E0CF910C94A31CC5
:101C9000AB01BC018FE090E00C94B41CAB01BC0123
:101CA00083E190E00C94B41C60E070E0CB010C94F4
:101CB0004E0E60E070E0CB010E94480E0C94540E72
:101CC00069EE7EEF80E090E00E94C01C60E082E060
:101CD00090E00E94A31C60E083E090E00E94A31CBF
:101CE000109236011092370110923801109239018A
:101CF00060E084E090E00E94A31C60E082E290E05B
:101D00000E94A31C60E085E090E00E94A31C60E0BC
:101D100086E090E00E94A31C6FEF87E090E00E94B5
:101D2000A31C40E050E0BA0188E090E00E94B41C9F
:101D300060E08DE090E00E94A31C40E050E0BA011A
:101D400088E190E00E94B41C60E087E190E00E948E
:101D5000A31C40E050E0BA018CE190E00E94B41C6A
:101D600060E070E080E290E00E94C01C40E050E043
:101D7000BA0188E190E00E94B41C0C94590E0C94B6
:101D8000600E682F8EE090E00C94A31C0E9407194F
:101D900060939601709397018093980190939901B5
:101DA00060939201709393018093940190939501B5
:101DB000089584B7806884BF84B7806884BF08951D
:101DC00081E008950C94E00E08950C94E40E0C94B8
:101DD000E40E0C94E70E0C94E40E0C94EB0E0C94B1
:101DE000E40E0E94D90E8DEA91E10E9421180E9412
:101DF000EF0E0C94ED0E0E94E50E0C94E40E0E9482
:101E0000C7110C9470030E94F4180E94AC120E9437
:101E1000FF0E0C94E90E5F926F927F928F929F92C9
:101E2000AF92BF92CF92DF92EF92FF920F931F93E8
:101E3000CF93DF93CDB7DEB72A970FB6F894DEBF06
:101E40000FBECDBF0E94C112C82E81110E94C60EC6
:101E500036E8832E31E0932E00E010E0502E802FE4
:101E60000E94EB115C01F401619071904F016826B2
:101E7000792661147104B1F40F5F1F4F063011050C
:101E800069F78FEF89838A831B820E94FB18816028
:101E9000782F9D838C8349815A816B818D810E942B
:101EA0008C033AC080919A0181FD0E94F411D12CDB
:101EB000EE24E394F12CC3018E219F21892B29F17B
:101EC0000E94E20E8823A9F0DE825F82AE20BF204E
:101ED00081E0AB2809F480E088870E94FB188160CC
:101EE000782F9A8789874E815F8168858A850E94CD
:101EF0008C03000F111FF801EA57FE4F808191817A
:101F0000E826F926F182E08207C0D394EE0CFF1C8C
:101F1000FFE0DF12D0CFB0CF81E0C11001C080E080
:101F20002A960FB6F894DEBF0FBECDBFDF91CF91DA
:101F30001F910F91FF90EF90DF90CF90BF90AF90E7
:101F40009F908F907F906F905F9008950E940B0FED
:101F50000E94C2140C948103CF93DF930E94D61089
:101F6000EC01811521E5920708F045C0811530E5A7
:101F7000930708F094C0883E910528F5803E9105AE
:101F800008F0F8C0883A910570F4853A910508F098
:101F90007CC08130910509F475C008F4E8C004974D
:101FA00008F0E8C0E4C08F3B910508F0E0C0C85AD3
:101FB000D0E0CC0FDD1FC555DF4F0990D881C02D73
:101FC000CE019464D8C0811540E2940758F481157D
:101FD00051E0950708F0CEC08D3E910508F4C7C0CA
:101FE0009065C9C0C11580E4D80708F4C0C0DF708F
:101FF000CE01906AC0C0811525E59207A8F481152D
:1020000034E5930708F095C0811543E5940708F07F
:102010007BC0811552E5950708F061C0D82FCC2709
:10202000CE01816F906AA7C0C11589E5D807A0F4D9
:10203000C11528E5D20708F082C0C11536E5D307DF
:1020400008F095C08C2F0E946A118F7190E0D82FF4
:10205000CC27CE0190628FC0C1154AE5D40708F4A1
:1020600074C0CE0190568115904208F080C08D2F2B
:102070008F710E946A11DD27D0628F71AE01582BDB
:10208000CA0179C081E090E076C0C55AD0E0C7525D
:10209000DF4F8881C82FD0E0CE0190646CC074E01F
:1020A000969587957A95E1F7282F23703C2F33700A
:1020B00081E090E002C0880F991F3A95E2F79C6892
:1020C000AC01522B9A019C2F9F709695969550E2E9
:1020D000959FE0011124C9018C2B9D2B4CC083706E
:1020E000992721E030E002C0220F331F8A95E2F7E2
:1020F0009C2F9695969580E2989FE0011124C22B23
:10210000D32BCE019C6837C08370992721E030E043
:1021100002C0220F331F8A95E2F79C2F9695969561
:1021200040E2949FE0011124C22BD32BCE019A6888
:1021300022C0D82FCC27CE01846F906A1CC0DC2F20
:10214000CC27CE01806F906A16C08C2F8F700E94B2
:102150006A1194E0D695C7959A95E1F7CF70D0E0D3
:10216000DC2FCC27D0699E01282BC90104C080E058
:1021700090E001C0CE01DF91CF9108952AE5829FC2
:10218000C0011124FC012FE0729FE00DF11D11240C
:10219000E60FF11DEE0FFF1FE459FF4F859194915B
:1021A00008950E94BE100E94AC0F089582389105D8
:1021B00069F1B0F48133910509F46DC048F48932B6
:1021C000910509F463C08A32910509F469C0089544
:1021D0008533910509F455C089339105B9F0089507
:1021E000833E910569F138F4803E9105B1F0823E5D
:1021F000910509F10895863E9105A9F1873E910563
:10220000B9F1843E910509F064C023C020914D02CC
:1022100020FD4FC021FD4DC0089580914D0280FDED
:1022200044C080914E0280FF44C080914D0284FDE5
:1022300042C083EE4DC080914D0282FF38C0F5CF81
:1022400080914D0282FD33C080914E0280FD31C0ED
:10225000ECCF80914E0281FF32C080914D0284FD0F
:102260002AC087EE35C080914D0283FF26C0F5CF8E
:1022700080914D0283FD21C080914E0281FD1FC0DF
:10228000ECCF80914D0285FD1CC01DC080914D0298
:1022900085FD19C016C080914D0286FD16C017C07D
:1022A00080914D0286FD13C010C089E311C082EEFB
:1022B0000FC080EE0DC080E00BC086EE09C084EE3A
:1022C00007C089E205C085E303C08AE201C081E35B
:1022D00090E0089590914D0292FF0DC0282F287133
:1022E000283019F4877F846006C0282F2471243099
:1022F00011F48B7F886093FF0DC0282F287128313F
:1023000019F4877E846106C0282F2471243111F4CA
:102310008B7E886120914E0220FF0DC0382F3871CE
:10232000383019F4877F816006C0382F3171313021
:1023300011F48E7F886021FF0DC0282F287128316D
:1023400019F4877E816106C0282F2171213111F493
:102350008E7E886194FD877E089580E008950C94B8
:10236000110E0E94C1128FE39CE90197F1F700C0A2
:1023700000000E94C11280E00E94EB1180FF04C0A7
:102380000E94AF110C94481908950C94B1110E9449
:10239000170E811102C00E94BF0E0E94220E809370
:1023A0009A010E942A0E90934E0280934D020E9441
:1023B000C5110E94260E682F70E080E090E00E9418
:1023C0000308609132017091330180913401909142
:1023D00035010C943B08E82FF0E0EE0FFF1FE55AA3
:1023E000FD4F808191810895089580EA8A95F1F7E3
:1023F000089500C008950C94F51108950C94FD11F2
:102400000C94FE110C94FD110C940212F894E82F18
:10241000E295EF70F0E031A9282F2F7081E090E075
:1024200001C0880F2A95EAF7982F9095932391ABD6
:1024300092A9892B82AB789408950F931F93CF9321
:10244000DF93CBEED0E089918F3F11F00E9406120E
:1024500080E0C13FD807B9F7CCEDD0E00BEE10E03B
:1024600089918F3F11F00E9406120C171D07C1F7CA
:10247000DF91CF911F910F910895BF92CF92DF927C
:10248000EF92FF920F931F93CF93DF938C01C62F90
:10249000D0E0CE0185519F4F6C01FC0190819F3FA0
:1024A00009F450C0B62EF894E92FE295EF70F0E0F1
:1024B00081A99F7021E030E001C0220F9A95EAF7D0
:1024C000822B81AB82A92095282322AB78940E948D
:1024D000F911ECEDF0E04BEE50E021E030E0E12CC2
:1024E000F12C61916F3F89F0A62FA295AF70B0E0FB
:1024F000D0968C9190E06F7002C0959587956A9503
:10250000E2F780FD02C0C90102C080E090E0E82A45
:10251000F92A220F331F4E175F0719F7F601808142
:102520008F3F11F00E94061261E0E114F10409F4FA
:1025300060E08B2D0E94FB11CC0FDD1FC00FD11F5F
:10254000F982E882DF91CF911F910F91FF90EF9078
:10255000DF90CF90BF9008950E941D128CE0EBE5B4
:10256000F2E0DF01982F1D929A95E9F7EFE4F2E08F
:10257000DF011D928A95E9F786E00E940C130C9406
:10258000FB02FF920F931F93CF93DF93CDB7DEB77C
:102590002C970FB6F894DEBF0FBECDBF8E010F5F34
:1025A0001F4F8CE0F80111928A95E9F7F12C6F2DFD
:1025B000C8010E943D12F394F6E0FF12F8CF4CE000
:1025C00050E0B8018FE492E00E94881CFF24F3944D
:1025D000009709F4F12C892B41F08CE0F801AFE46D
:1025E000B2E001900D928A95E1F72F2D46E06BE560
:1025F00072E08FE492E00E940D130E94FD028F2D85
:102600002C960FB6F894DEBF0FBECDBFDF91CF91F1
:102610001F910F91FF9008950895FF920F931F93BC
:10262000CF93DF93F82E092F162FD72FC42F2223F5
:1026300049F081E080939D010E94FB1890939C01DA
:1026400080939B0180919D018823D9F080919B010B
:1026500090919C010E941319059798F0EF2DF02F8F
:10266000A12FBD2F80E090E04C2F50E084179507FC
:1026700034F4219131912D933D930196F7CF10922F
:102680009D01DF91CF911F910F91FF9008950E94BE
:1026900062190E94030F0C9473190E94E9180E949A
:1026A0005B190E94F10E0E9447130E9481190E943B
:1026B000FB0EFBCF8091A40180FF06C060916900F2
:1026C00070E0660F771F26C081FF04C0609169002B
:1026D00084E005C082FF07C06091690088E0689FC0
:1026E000B001112417C09091A3019923D1F06091FA
:1026F0006800961788F72091690088E0289F90016C
:102700001124929FA001939F500D112470E0CA01E3
:102710000E945A1C6038710540F46115710519F466
:1027200006C068E070E0862F08958FE7089581E085
:1027300008958091A40180FF08C06091650070E059
:10274000759567957595679521C081FF06C0609165
:10275000650070E07595679519C082FF04C06091AF
:10276000650070E010C09091A201992399F06091EA
:1027700064009617A0F780916500899FC00111241D
:1027800070E00E945A1C6038710540F461157105B3
:1027900019F406C061E070E0862F08958FE7089570
:1027A00081E008958D3E21F40E945A13819504C062
:1027B0008E3E29F40E945A138093A80108958F3EFB
:1027C00021F40E945A13819504C0803F29F40E948D
:1027D0005A138093A7010895893F19F40E94991311
:1027E00005C08A3F31F40E94991381958093A90115
:1027F00008958B3F21F40E949913819504C08C3F6A
:1028000029F40E9499138093AA0108959FE0980FDC
:10281000983078F421E030E0A90102C0440F551F40
:102820009A95E2F7CA019091A601892B8093A6019F
:1028300008958D3F21F48091A40181600BC08E3FEB
:1028400021F48091A401826005C08F3F29F480911A
:10285000A40184608093A40108958D3E39F4909181
:10286000A80197FF35C01092A80159C08E3E29F4E7
:102870009091A8011916BCF32BC09091A7018F3E2F
:1028800029F497FF25C01092A70149C0803F19F491
:102890001916CCF31DC09091A901893F29F419168E
:1028A000BCF41092A9013BC08A3F19F497FF10C0F5
:1028B000F8CF8B3F39F49091AA0197FF09C010928D
:1028C000AA012DC08C3F21F49091AA011916BCF3E6
:1028D0009FE0980F983080F421E030E0A90102C019
:1028E000440F551F9A95E2F7CA0180959091A60171
:1028F00089238093A60113C08D3F21F48091A40108
:102900008E7F0BC08E3F21F48091A4018D7F05C086
:102910008F3F29F48091A4018B7F8093A401809143
:10292000A701811106C08091A801811102C01092F7
:10293000A3018091A901811106C08091AA01811192
:1029400002C01092A20108950E94FB182091A701D5
:10295000211104C02091A801222321F09093A1010C
:102960008093A0012091A901211104C02091AA0106
:10297000222321F090939F0180939E0185EA91E0AC
:102980000C944218EF92FF920F931F93CF93DF9313
:1029900000D000D000D0CDB7DEB786E0E5EAF1E0A8
:1029A000DE01119601900D928A95E1F7E090A70162
:1029B000F090A8010091A9011091AA011092A7011D
:1029C0001092A8011092A9011092AA01E11003C06F
:1029D000FF2009F45DC08091A0019091A1010E94A7
:1029E0001319AC019091A301992339F020916A0049
:1029F00030E02417350758F04BC020916B008AE077
:102A0000289F900111242417350718F041C09F3FDB
:102A100019F09F5F9093A301EE2061F00E945A137A
:102A20001E1414F09FEF01C091E0989F902D112487
:102A30009093A701FF2061F00E945A131F1414F015
:102A40009FEF01C091E0989F902D11249093A801D1
:102A50003091A7013323E1F02091A8012223C1F096
:102A600045EB3403C0011124992319F09093A70179
:102A700003C081E08093A70135EB2303C00111243B
:102A8000992319F09093A80103C081E08093A801D5
:102A9000011103C0112309F45DC080919E01909142
:102AA0009F010E941319AC019091A201992339F062
:102AB0002091660030E02417350758F04BC0209174
:102AC00067008AE0289F900111242417350718F029
:102AD00041C09F3F19F09F5F9093A201002361F0D6
:102AE0000E949913101614F09FEF01C091E0989F77
:102AF000902D11249093A901112361F00E94991344
:102B0000111614F09FEF01C091E0989F902D1124B1
:102B10009093AA013091A9013323E1F02091AA01F9
:102B20002223C1F045EB3403C0011124992319F08D
:102B30009093A90103C081E08093A90135EB2303A1
:102B4000C0011124992319F09093AA0103C081E0D8
:102B50008093AA018091A70181110BC08091A801E7
:102B6000811107C08091A901811103C08091AA0140
:102B700081110E94A414EB82FC820D831E8386E0E7
:102B8000FE013196A5EAB1E001900D928A95E1F738
:102B900026960FB6F894DEBF0FBECDBFDF91CF9162
:102BA0001F910F91FF90EF900895E5EAF1E086E024
:102BB000DF011D928A95E9F71092A3011092A201FC
:102BC0001092A4010895CF93DF93EC01FB01828161
:102BD000882309F43CC1C430FDE5DF0760F4CB3F36
:102BE0009CE5D90788F49E0122503C4524313105EB
:102BF00008F02EC109C0C236EDE5DE0729F0C63A5D
:102C0000FDE5DF0709F024C10E942A0E90934E02D1
:102C100080934D02C1318CE5D80709F4C6C008F095
:102C200042C0C930ECE5DE0709F49BC000F5C530B1
:102C30008CE5D80709F485C078F4C330ECE5DE07ED
:102C400009F478C008F07AC0C230DC4509F0F5C05C
:102C500080914D028160EFC0C7309CE5D90709F42F
:102C600078C008F07AC080914D028061E4C0CD3018
:102C7000FCE5DF0709F487C058F4CB309CE5D907A1
:102C800009F479C008F07BC080914D0288606FC064
:102C9000CF30FCE5DF0709F480C008F082C08091E6
:102CA0004D02877FC8C0CE3F9CE5D90709F471C0AB
:102CB00000F5C531FCE5DF0709F485C068F4C331D0
:102CC0009CE5D90709F475C008F095C00E94AB07D0
:102CD00080914D028F77AFC0CC3FFCE5DF07A9F1B3
:102CE00008F054C0CB3FDC4509F0A7C080914E02EC
:102CF00040C0C230EDE5DE0709F489C058F4C115C3
:102D00008DE5D80709F45AC008F069C080914E02D9
:102D100082602FC0C236EDE5DE0709F47CC0C63AFA
:102D2000FDE5DF0709F481C0C330DD4509F085C04A
:102D300080E06EC080914D0282607DC080914D0226
:102D400016C080914D02886076C080914E028260EC
:102D50004FC080914D0280626EC080914D028064B0
:102D60006AC00E94AB0780914D02806864C0846095
:102D700062C081603DC080914D028E7F5CC08091B9
:102D80004D028D7F58C080914D0216C080914E0239
:102D900018C080914E028D7F2BC080914D028F7E96
:102DA0004AC080914D028F7D46C080914D028F7B3D
:102DB00042C080914D02877F8B7F3DC080914E0243
:102DC0008D7F8E7F15C080914D0282FB222720F9D6
:102DD00091E0922790FB82F990FB83F92CC08091BF
:102DE0004E02982F909591708E7F892B90FB81F9E0
:102DF00080934E0222C00E94AB0780914D0287FB58
:102E0000222720F991E0922790FB87F914C081E0F6
:102E10000E94C10E12C080914D0284FB222720F92E
:102E200091E0922790FB84F906C080914D02982F83
:102E3000909590FB80F980934D0280914D02909186
:102E40004E020E943B0E0E94AB0780E001C081E071
:102E5000DF91CF910895CF93DF9386319C4541F563
:102E6000EB010E942E0D982F8A81209162003091F3
:102E70006300882379F09A7A81E009F480E08093F6
:102E8000AB01911102C069E201C065E3C9010E9472
:102E9000BE180AC08091AB01811102C069E201C075
:102EA00065E3C9010E94C0180E94700D80E001C056
:102EB00081E0DF91CF9108950F931F93CF93DF931C
:102EC000C42FD22FFC0182818823C9F04093AE0128
:102ED0000E94FB189093AD018093AC0180E28C0FAF
:102EE000883008F057C0C77081E001C0880FCA95CC
:102EF000EAF7DF91CF911F910F910C940E0580910D
:102F0000AE01481330C08091AC019091AD010E9498
:102F10001319883C910538F510E21D0FCD17B9F053
:102F200080E28C0F883040F4C77081E001C0880FC8
:102F3000CA95EAF70E941505183028F581E09D2F03
:102F4000977001C0880F9A95EAF70E940E05802FAE
:102F50000E9405051830F0F4D77081E001C0880F99
:102F6000DA95EAF70AC080E28C0F883098F4C770CF
:102F700081E001C0880FCA95EAF7DF91CF911F91D8
:102F80000F910C941505802FDF91CF911F910F9118
:102F90000C940505DF91CF911F910F9108950F9328
:102FA0009C01CB01243F4CE5340731F188F4293DE5
:102FB000FCE53F07D9F02A3D4CE5340779F1283D7F
:102FC0003C45A9F506E221EE41EE68ED7CE52BC01B
:102FD000263FFCE53F07E1F0A8F0273F3C4539F5E7
:102FE00007E225EE46EE67EF7CE51DC007E225EE21
:102FF00045EE69ED7CE517C006E221EE40EE64EF98
:103000007CE511C007E225EE44EE65EF7CE50BC0E0
:1030100006E221EE42EE66EF7CE505C008E221E023
:1030200045EE6AED7CE50E945C1780E008C0FC017B
:103030008281882319F01092AE0101C081E00F91C6
:1030400008959093F3008093F20008959093B40153
:103050008093B3010895E091B301F091B4013097EA
:1030600021F00190F081E02D099480E00895E09135
:10307000B301F091B401309721F00280F381E02D8B
:1030800009940895E091B301F091B401309739F0BB
:1030900022E0DC012C930480F581E02D0994089551
:1030A0002091B1013091B2012817390771F0909346
:1030B000B2018093B101E091B301F091B401309776
:1030C00021F00680F781E02D099408952091AF0149
:1030D0003091B0012817390771F09093B0018093B7
:1030E000AF01E091B301F091B401309721F0008479
:1030F000F185E02D09940895FC01329697E080E077
:10310000915029F021912223D9F38F5FF9CF0895AF
:10311000662349F0FC01329608962191621729F046
:10312000E817F907D1F780E0089581E008959C0140
:10313000FC0132969FEF80E04191461789F09F3F56
:1031400019F4411101C0982F8F5F8630A9F79F3F76
:1031500039F0F901E90FF11D97FDFA9562830895A1
:1031600008959C012A5F3F4FFC014281461301C034
:103170001282019682179307B9F708950C94971855
:103180000C94B118029626E0FC0111922A95E9F7F9
:10319000089508950C94C9180C94CA180C94C91871
:1031A0000C94C9180C94C918CF930E94D0180E948F
:1031B000C1120E94CE18C0E08C2F0E94EB11892B07
:1031C00029F4CF5FC630C1F780E001C081E0CF9124
:1031D000089508958091B70181110C9461030895B9
:1031E0000E94AB070C9465038BE083BF8AEF8CBF12
:1031F00082E089BF08952FB7F8948091670290917B
:103200006802A0916902B0916A022FBF08952FB79A
:10321000F8946091670270916802809169029091C0
:103220006A022FBF08959C014FB7F89480916702FE
:1032300090916802A0916902B0916A024FBF821B0F
:10324000930B089578941F920F920FB60F9211244A
:103250008F939F93AF93BF93809167029091680281
:10326000A0916902B0916A020196A11DB11D8093DF
:10327000670290936802A0936902B0936A02BF91BB
:10328000AF919F918F910F900FBE0F901F90189547
:1032900098E088E10FB6F894A89581BD0FBE91BD66
:1032A000A895F894D8E0CEE528E3299320E0299367
:1032B00014BEFFCF08950E94FB189093B60180932F
:1032C000B50108950E943F1C8B9A80E0815041F027
:1032D000A895EFE9FFE03197F1F700C00000F6CFC5
:1032E0008B98789408950E94671A0E9426182FEFF1
:1032F00080E792E0215080409040E1F700C000005C
:10330000089580919202882389F0109292020E947F
:10331000FB189093B6018093B5018091B701882383
:10332000D1F11092B7010E94F01811C08091B7013D
:10333000811111C08091B5019091B6010E941319BD
:10334000069728F081E08093B7010E94EA188091E7
:10335000B701882301F10E94EA180E94D41888233B
:1033600039F1F89421B3939A822F8C6081BB92B388
:103370008CE0982792BB3FE748E391E03150404012
:103380009040E1F700C0000092B3892782BB21BBC7
:103390009398789408950E94481B809198028823FE
:1033A00029F08091760284FD0E94A60F0C940E1ADB
:1033B000089580914C02089508959091BD0198134D
:1033C00007C02091BB013091BC0126173707A9F037
:1033D0008093BD017093BC016093BB018093B801E1
:1033E0007093BA016093B9018091AF0284FF05C068
:1033F00063E088EB91E00C94441B0895BC0184E0E9
:103400000C94DD19BC0183E00C94DD192091AF020E
:1034100024FF03C066E00C94441B0895CF93DF9310
:10342000CAE0D0E08091760284FF18C08091C90183
:103430009091CA019817E1F028E0829FC001112401
:1034400068E085539E4F0E94401B8091C90190E027
:1034500001968F7099278093C9010AC00E94481B6A
:103460008FE99FE00197F1F700C000002197D1F6A6
:10347000DF91CF910895CF93DF93EC01A091CA0122
:10348000B0E0CD0101968F7099272091C9012817CE
:1034900079F093E0AA0FBB1F9A95E1F7A553BE4FB1
:1034A00098E0FE0101900D929A95E1F78093CA0190
:1034B0000E94481B0E940E1A88E0FE01A1ECB1E0B8
:1034C00001900D928A95E1F7DF91CF9108958CE6F6
:1034D00090E00895FC01808180768032A1F58181A1
:1034E000813061F484819581892B69F581EC91E0CB
:1034F000909394028093930288E00895823041F47F
:103500008BE492E0909394028093930281E008957B
:103510008A3021F4838180934B0215C0893099F45D
:10352000828193818115924081F484819581892BD8
:1035300061F481E08093C001868197819093BF01FF
:103540008093BE0102C080E008958FEF089520911E
:10355000BE013091BF01232B71F02091C0012130B9
:1035600051F4FC01808180934C021092BF011092B3
:10357000BE0181E008958FEF08950895FC019381C5
:103580009330D9F068F4913081F0923009F054C052
:1035900080E291E090939402809393028BE30895EC
:1035A000913221F1923291F147C08BE591E09093F5
:1035B00094028093930282E108958281813071F0B8
:1035C00028F08230C9F58DE691E00AC081EA91E0E9
:1035D000909394028093930284E0089587E891E0A9
:1035E000909394028093930288E1089582818823C6
:1035F00029F0813009F58BE491E002C082E391E08B
:10360000909394028093930289E008958481958138
:10361000009751F0019781F485EA91E0909394022C
:10362000809393028BE7089580E292E09093940256
:103630008093930280E4089580E008951F93CF93D0
:10364000DF93162FEA01288124FF05C0398128E87D
:103650002327298302C02AE52883212FFC01CE01DC
:103660000296DC0131913D9321501216DCF3612F5B
:103670000E9464011C5F1883DF91CF911F91089510
:1036800046E752E00C941E1B4FEA52E00C941E1BBE
:10369000CF93DF9360919502635067FD93C0809153
:1036A0009102CCE0D0E0C81BD109C756DD4F809114
:1036B0009002803120F4CE010E94BD1A81C08D326B
:1036C00009F06EC0683009F07BC083EC80936B0218
:1036D0008AE58093790010928F028881807621F0AC
:1036E000CE010E946A1A49C09A811092740289819F
:1036F000811106C01092750224E732E082E038C0E2
:10370000853019F49093960230C08630A1F48B81F5
:10371000813041F0823031F0833021F0813211F07C
:10372000823221F4CE010E94BE1A01C080E090E4F2
:1037300090938F0222C0883089F0893019F49093D9
:10374000980213C08A3069F08B3079F48BE480934F
:1037500077028093B0028093830207C028E932E0A9
:1037600002C024E732E081E003C024E732E080E0D9
:10377000309394022093930209C08F3F39F49881CB
:1037800097FD8E8190E890938F0207C09F819111E1
:1037900004C09E81981708F4892F8093780010C088
:1037A00080918F0287FF0CC0CE010E94A71A8F3F25
:1037B00021F48EE18093790003C08111109278008A
:1037C000109295028091790084FF4CC0809178001E
:1037D0008F3F09F447C0C82F893008F0C8E08C1B20
:1037E0008093780090916B0288E8892780936B0220
:1037F000CC2359F1809193029091940220918F02F1
:1038000026FF12C0ABE6B2E02C2FAC014B56524063
:10381000FA01EA0FFB1FE4911196EC9311972150E6
:1038200011962111F5CF08C0ECE6F2E0DC012C2F57
:103830003D9131932150E1F701962FEF2C0F820F2C
:10384000911D90939402809393026C2F8CE692E0EA
:103850000E946401CC5FCC3019F08FEF8093780028
:10386000C093790084E190B39C7031F48150D9F712
:103870001092960210928E02DF91CF910895CF930D
:10388000DF9385B7886085BF8BB780688BBFC6E73D
:10389000D2E08BE48983AFEAB2E011968C93119762
:1038A000E2E8F2E081838AE588838C938083DF916C
:1038B000CF91089597FB072E16F4009407D077FD5B
:1038C00009D00E94741C07FC05D03EF490958195A8
:1038D0009F4F0895709561957F4F0895EE0FFF1FDC
:1038E0000590F491E02D0994AA1BBB1B51E107C080
:1038F000AA1FBB1FA617B70710F0A61BB70B881F80
:10390000991F5A95A9F780959095BC01CD0108950E
:10391000FB01DC0104C08D910190801921F441501C
:103920005040C8F7881B990B0895E199FECF9FBBC3
:103930008EBBE09A99278DB30895A8E1B0E042E0EC
:1039400050E00C94C81C262FE199FECF9FBB8EBB84
:10395000E09A01970DB2021631F02DBB0FB6F89424
:10396000E29AE19A0FBE08950396272F0E94A41CA5
:103970000E94A31C252F0E94A41C242F0C94A41C7D
:103980000196272F0E94A41C0C94A31CDC01CB01E0
:10399000FC01E199FECF06C0FFBBEEBBE09A319679
:1039A0000DB20D9241505040B8F70895F894FFCFF2
:1039B000C8007C01280850011E0A1401D9193B1ABD
:1039C000061A021AFE19DC19FF5AE200E900EA00A1
:1039D000B500B600B700CD008301CC008A0192018A
:1039E00094012102230224022502260227022A0230
:1039F000B300B4006F007000818283E200E900EA46
:103A000000B500B600B700CD008301CC008A01925A
:103A10000194012102230224022502260227022A00
:103A200002B300B4006F0070008182839091929382
:103A300094950605016061626364073435363797F3
:023A40009600EE
:00000001FF
